:100000006D28FF3FFF3FFF3FA53003138312FA0027
:10001000FA0B0828000000000800031383123608BA
:1000200083169B009C131C141A08F000080003138D
:1000300083123708F0000130F100F2017008031953
:100040002628F10DF20D7110FF3F1F287108BA002C
:10005000360884000008F0007108F00570080130CF
:10006000031D0030F0003908F00603195128380844
:10007000003C03183F2804200420B8033728360822
:1000800084000008F0003A08F00570080130031DF4
:100090000030F0003908F00603195128FF30F00055
:1000A0000800F00108000000031383169C1C5A2866
:1000B000000054288312360883169B0083123708E9
:1000C00083169A009C131C158B1355309D00AA3083
:1000D0009D009C148B171C110800031383168601C6
:1000E0008312860107309F00F0308316850083124B
:1000F00085013F30A0000630A1005B30A2004F30E8
:10010000A3006630A4006D30A5007D30A600073046
:10011000A7007F30A8006F30A9007730AA007C309C
:10012000AB003930AC005E30AD007930AE007130DC
:10013000AF00B6010D2070088312B40070080F3CA8
:100140000318A328B4013408203F84000008860067
:1001500034088500B6010D2070088312B4007008C1
:100160000F3C0318B428B4013408203F8400000871
:100170008600340885000530B6000430B700013031
:10018000B800B901172070080319C8280130B5005C
:1001900035080319DE280530B6000430B7000130F9
:1001A000B8000130B900172070080319DE28B40A1E
:1001B000B6013408B70053208312B501AA28DF28FE
:02400E00583F19
:00000001FF
